:030000000219FDE5
:03000B000200AA46
:03002B0002016669
:03005B000202FCA2
:030073000202E2A4
:1000800002030406080C10182030406080040608A3
:100090000C10182030406080A0C000070F1F3F0DDB
:1000A0000D0403060D0503030202C2AFC0D0C0E079
:1000B000206217E5256002E473E525F4F58A758B67
:1000C00000D262D0E0D0D0D2AF3285268AC262E5BB
:1000D00026F46036306803207210758B00D0E0D0B3
:1000E000D0C290C287C291D2AF32C290C287C291B1
:1000F000206E0D20660A7401D5E0FDE57EF4529075
:10010000758B00D0E0D0D0D2AF32758A00C28DD2CC
:1001100062210001B9306805206602D29001B93031
:100120006805206602D28701B9306805206602D2D0
:100130009101B9D29630680A2066077405D5E0FDB2
:10014000D29001B9D29430680A2066077405D5E0D0
:10015000FDD28701B9D29530680A2066077405D5AB
:10016000E0FDD29101B9C2AFC2AD53E6EFC0D0C03D
:10017000E0D2D3D2AFC2CEE52A6007207449152A57
:1001800021C77800790020742EE580307E01F4309C
:10019000E60278FF53DACF207E0343DA20307E0375
:1001A00043DA10C2D8C271E580307E01F430E60235
:1001B00079FFC3E89970CB306103752A402074033E
:1001C000752A40885FD27020740DE52B6004152BD2
:1001D00021D743DA01C2D820700221EAA85F20614A
:1001E00002C27020740221E888227882B604038556
:1001F0002224C3E52594404002D26420CF0AD0E0F7
:10020000D0D043E610D2AD32C2CF053A7802E52A0B
:100210006005307402152AC3E55F940140057562DC
:10022000004134756300756C00E5622401F562508D
:10023000037562FF7982B7020D306D1DC3E522940C
:10024000324016854D227982B7030E306D0BC3E51F
:100250002294324004798E8722C3E52395226008D8
:100260004004152341680523D8CA056CE56C70026B
:10027000156CD56D63756D017805C3E56C956E40A1
:1002800057C3E56C956F50087801756D0302029CA9
:10029000C3E56C957050057801756D01C3E56595F2
:1002A00024401E7982B7040241CD206D1485246557
:1002B000E56C046003856E6C756D0175233C02026C
:1002C000D8E5652850057565FF41CDF565E5650400
:1002D00070067563FF756CFFD0E0D0D043E610D296
:1002E000AD32C2AFC0D053E67FC260759100855673
:1002F00094855795759104D0D0D2AF32C2AF53E6F2
:10030000EFC2ADC0D0C0E0C0F0D2D3D2AFA8FBA93D
:10031000FCC2D8307102616353DACF207E0343DA26
:1003200010307E0343DA20D271E580307E01F42064
:10033000E602613A88278928A14853DACF207E0354
:1003400043DA20307E0343DA10C2D8C2713074021F
:10035000A1347800E580307E01F430E602A13488D3
:100360005FA11C53DACF207E0343DA20307E0343A3
:10037000DA10C271206102813C53DACF207E034340
:10038000DA10307E0343DA20C2D8D271885A895BF2
:10039000C3E89558F8E99559F97B007E087A00C3BF
:1003A000E8948CE994005005755E00812E882178D0
:1003B000A2E6A8216055C3E894C8E994005008E477
:1003C000D2E4FB7A0A8109C3E89468E994015008F1
:1003D000E4D2E3FB7A0F8109C3E894D0E994025098
:1003E00008E4D2E2FB7A1E8109C3E894A0E99405EF
:1003F0005008E4D2E1FB7A3C8109C3E89498E9947F
:10040000085008E4D2E0FB7A787E00C3E8955CFCF3
:10041000E9955DFD30E70AECF42401FCEDF43400CD
:10042000FD755E00C3EC9AED9E5003755E01885C1D
:10043000895D855A58855B597802A11CC3E89527C8
:10044000F8E99528F9307C02A100307B02A1003048
:100450007A0281F9207502815FE9FDE8FC817EE97D
:10046000C313F9E813F830790281F9E9C313F9E805
:0E04700013F830780281F9E9C313FDE813FC9C
:10047E0020612CC3EC941CED940240028195ED702A
:10048E001EC3EC94C850180529E52970021529C31E
:10049E00E529940A5002A134755F00D270A134E5AB
:1004AE0029600215297400207F037896E624FAFE4F
:1004BE00E43400FFC3EC9EFCED9FFD5006780079FE
:1004CE0000A100C3EC94FFED9400400678FF790084
:1004DE00A100EC8575F0A4C5F0A2F733F8790040C1
:1004EE000302051C78FF790002051CE9C313F9E825
:1004FE0013F8307C0EE9600278FFC3E81338F8E495
:10050E003400F9C3E894FFE99400400278FF885F55
:10051E00D270206102A134741FF4552F4BF52FC2F7
:10052E0074EB7002D274752A40307403752A0A3047
:10053E006102A14820740353DAFE207403752B2048
:10054E00D0F0D0E0D0D0D2AD43E610327901020522
:10055E00787903020578790A020578791E02057802
:10056E00796402057879C80205787817E4D5E0FD3C
:10057E00D8FAD9F6227A147B7802059F7A107B8CF2
:10058E0002059F7A0D7BB402059F7A0B7BC802058C
:10059E009F7902B27DE4D294D5E0FDD287D5E0FDFD
:1005AE00C287D5E0FDC294D5E0FDD290E576D5E0C8
:1005BE00FDC2907496D5E0FDD9D9EAF8D5E0FDD804
:1005CE00FBDBCED29422C37C007D0075F00005F0DB
:1005DE00EA33FAEB33FB50F6EB13FBEA13FAC3E9FB
:1005EE00FFE8FEE89AF8E99BF95004EFF9EEF8B34C
:1005FE00EC33FCED33FDD5F0DFEDF9ECF822E889B4
:10060E00F08A20D2D4F8A9F07B0030F70B7BFFF4F0
:10061E002401F8E9F43400F9E88520F0A4ADF0F8EF
:10062E00E98520F0A4AFF0FEED2EF974003FFA7CC0
:10063E0004C3EA13FAE913F9E813F8DCF48BF0308B
:10064E00F70AE8F42401F8E9F43400F9E889F0C275
:10065E00D4F8A9F0227882B60403020702C3E55F3C
:10066E009419401EE52D54067018206D36780579C4
:10067E0094E7146007780A1460027812C3E5419873
:10068E00401F306D09856765756CFF756D0185229C
:10069E0024E4F545F546F547F548F549C26D0207E0
:1006AE0002D26D7994E7147013E523F43333F91302
:1006BE00F8E9540104F9E854FE0206F6E714147042
:1006CE0014E523F4333333F913F8E9540304F9E84A
:1006DE0054FC0206FEE523F433333333F913F8E901
:1006EE0054070404F9E854F8C39440F8E99400F967
:1006FE008845894622C3E54113F9E54013F8C3E561
:10070E004598F8E54699F9500CC3E89480E994FFB2
:10071E00401602073AC3E8947FE99400500302079B
:10072E003A787F790002073A788079FF884A894BB8
:10073E0022E54A2547F8E54B3548F9854B20E4304C
:10074E000701F43549FA30E709C3EA94F04015027F
:10075E000778C3EA940F500302077878FF79FF7A7F
:10076E000F020778780079007AF0C3E5249564507B
:10077E000AC374019524500B020796E54B20E70E31
:10078E00020796E54B30E706884789488A49227862
:10079E00A4E6FAC3E54A33F8E54B33F9D10CE93058
:1007AE00E70BC3E89480E994FF4013E1D0C3E894CB
:1007BE007FE994005002E1D0787F7900E1D0788013
:1007CE0079FFE820E715C3E52398F84009C3E894BC
:1007DE000140030207F778010207F7E8F424012528
:1007EE0023F840030207F778FF884C2278A5E6FA33
:1007FE00A848A94912060CE930E70CC3E89401E9B0
:10080E0094FF401602082CC3E894FFE994005003AD
:10081E0002082C78FF790002082C780179FFE92074
:10082E00E715C3E54C98F84009C3E894014003026C
:10083E0008537801020853E8F42401254CF84003CC
:10084E0002085378FF88242278FFC26420693D2075
:10085E006A12D264C3E541940A4009C3E525944067
:0F086E005002C26479A1E76023E541601F74FF67
:10087D008541F0848539F0306A0375F005A4F8C51B
:10088D00F0600278FFC3E895675002A8678866227A
:10089D00C3E5409440E5419401E56650031401AE73
:1008AD00046002F566227883E6F520120F4C75E898
:1008BD009012055A75E890E5E820ECFBA8BDA9BE9D
:1008CD00120FE6757180757202C3740213FD748088
:1008DD00606613FC74802CFC74023DFDECFAEDFB9C
:1008ED00C3E89AE99B4014E5712480F571E57234F3
:1008FD0002F572EA2CFAEB3DFB80E5AE71AF72C3E7
:10090D00E57213F9E57113F8C3E913F9E813F87AF1
:10091D0003C3E913F9E813F8DAF7AA201A70097579
:10092D0071007572000209451AEA6008EE28FEEFA3
:10093D0039FFDAF88E718F722275E890227883E68E
:10094D00FFE5E820ECF7A8BDA9BE0573C3E57394D8
:10095D00084052757300E9FA79A0E76044EA700720
:10096D00E574601B020980C3E895746010E574504E
:10097D0006600C1402098C0460F902098CE574F50B
:10098D0074C39467401B7564C0C3940440137564AD
:10099D0080C39404400B756440C394044003756494
:1009AD000075BB0A22EFC39401601F7480601BC3E6
:1009BD00E894FFE994035012C3E89571E9957250DC
:1009CD0009E564600C15640209DEE564F460020556
:1009DD0064A864C3E524985002A824C3E895654033
:1009ED000AA865E565F4600385656488258826E5B4
:1009FD0073B4070375BB1022743279A687F0A4C5B2
:100A0D00F0A2F733F8C3E895644002A86488228801
:100A1D0024882588268867227540007541F022C2FA
:100A2D00AF75C820A8CCA9CDAA3A30CF010A75C898
:100A3D0024D2AFAB3BAC3C883B893CC3E89BF8E987
:100A4D009C206908F93067026141419EAD3D8A3DA8
:100A5D00F9EA9DFA600478FF79FFAE3EAF3F8B3E19
:100A6D008C3FC3EC9FFCC3E99CF542A83BA93CC35A
:100A7D00E89EF8E99FF9C3E54113FBE54013FAE859
:100A8D002AF540E93BF54150067540FF7541FF41A0
:100A9D00E8AA40AB41AC40AD417E047F02C3EB946C
:100AAD000440021E1FC3EB940840021E1FC3ED132A
:100ABD00FDEC13FCDEF7C3EA9CFAEB9DFBEF60093E
:100ACD00C3E913F9E813F8DFF7EA28FAEB39FB8AE3
:100ADD00408B4150067BFF8B408B41C3EB94025002
:100AED0002D2673069047F0361137892E6FFC3E594
:100AFD0037948240110FC3E53794A040010FC3EF27
:100B0D00940640027F057E04E541C4540FF9E5418A
:100B1D00C454F0F8E540C4540F28F8C3E89EFAE930
:100B2D009400FB4009C3EA9402EB940050047A024E
:100B3D00E4FB618DAA40AB41EBC4FEEAC4540F4EF9
:100B4D00FCC3EA9CFAEB9400FBC3E813C313F8EA69
:100B5D0028FAEB3400FB8A408B41C3EB9402400230
:100B6D00C2677804EBC4FE7B00EAC4540F4EFAC38F
:100B7D00EA98FA4005C3940250027A027892E6FF91
:100B8D00306002618D855256855357D26043E680A1
:100B9D00C3E49AF8E49BF93067028127E8FAE9FB90
:100BAD00D3E913FDE813FC88528953C3EF94036016
:100BBD0038EF20E00DE82CF8E93DF9ECFAEDFB02F9
:100BCD000BE2E828F8E939F9C3E82402F8E9340022
:100BDD00F97AFE7BFFC3EF9403400E8A548B558840
:100BED004E894F8C508D51815B885489558A4E8B1F
:100BFD004F8C508D51306920C3E53394034019E576
:100C0D0042A2E713F8E555F4240138400B20E7081C
:100C1D007554FFF42401F555815BE8FAD3E813FC14
:100C2D008852C3EF94036020EF20E007E82CF8EC26
:100C3D00FA8147E8282402F87AFEC3EF94034008AE
:100C4D008A54884E8C50815B88548A4E8C50E56B4B
:100C5D00C3335002646BF56B3060028165753402ED
:0F0C6D00D26043E680E52D54066026A840A941D9
:100C7C00C3E913F9E813F8C2AF53E67F759100C3CB
:100C8C00E498F594E499F595759104D26043E68067
:100C9C00D2AF22D265754400752000306B037520ED
:100CAC0040020CBED265754400752040306B037554
:100CBC002000D2AF7801206722E52D54066002C2D5
:100CCC0065C3E54194054013780294054008780308
:100CDC00940540027806306902780A206019E544D0
:100CEC00601530690AC3E53394034003D53406D24A
:100CFC00AFD26CA18F916DD2AF0000C2AF2067262E
:100D0C00E541C3FB940F40027B0FEB2405307301CC
:100D1C0023306A02742820620123F9306902798237
:100D2C00E58BC39940B50544E59B5440B52002A121
:100D3C007930690A08C3E8940A40010881E7206504
:100D4C000281BEC26553E67F7591003067107594C1
:100D5C00007595FE759104D26043E68081BEAE406D
:100D6C00AF41C3E49EF594E49FF595A160C3E533D0
:100D7C009402500281BE30650281BED802A18D81E1
:100D8C00E7C26C53E67F7591008554948555957533
:100D9C009104854E56854F57D26043E680D2AFE51D
:100DAC002D54066008206A020533020DC9306C0D03
:100DBC00206B0A2065071581158102162422780004
:100DCC003064053065027801E53775F007A4F9E564
:100DDC00F028F5F0E9A2F013A2F113A2F213F53703
:100DEC00C394785003753778C3E53795384008D2EB
:100DFC0066C290C287C291306002C103855056858D
:100E0C005157D26043E68022207D11C2AF75430258
:100E1C00D294C296D2AF759F34020FE3C2AF754322
:100E2C0002D294C295D2AF759F34020FE330724355
:100E3C00207D20C2AF754303900144757E10C29192
:100E4C00D295306204D287C157C294D2AF759F3508
:100E5C00020FE3C2AF754303900144757E10C2903C
:100E6C00D296306204D287C177C294D2AF759F32CA
:100E7C00020FE3207D17C2AF75430390011FC2918F
:100E8C00306202D287D2AF759F35020FE3C2AF75C5
:100E9C00430390011FC290306202D287D2AF759F7C
:100EAC0032020FE3207D11C2AF754304D296C29576
:100EBC00D2AF759F32020FE3C2AF754304D295C215
:100ECC0096D2AF759F35020FE3307243207D20C25E
:100EDC00AF754305900133757E40C287D294306262
:100EEC0004D290C1F3C296D2AF759F34020FE3C205
:100EFC00AF754305900155757E20C287D294306240
:100F0C0004D291E113C295D2AF759F34020FE32046
:100F1C007D17C2AF754305900115C287306202D2AE
:100F2C0090D2AF759F34020FE3C2AF7543059001A9
:100F3C0029C2873062EBD291D2AF759F34020FE396
:100F4C00207D11C2AF754306D295C294D2AF759F66
:100F5C0035020FE3C2AF754306D296C294D2AF7579
:100F6C009F32020FE3307242207D20C2AF754301E5
:100F7C00900155757E20C290D296306204D291E1D8
:100F8C008FC295D2AF759F32020FE3C2AF7543018A
:100F9C00900133757E40C291D295306204D290E1BB
:100FAC00AFC296D2AF759F35E1E3207D16C2AF7507
:100FBC004301900129C290306202D291D2AF759F49
:100FCC0032E1E3C2AF754301900115C29130620268
:100FDC00D290D2AF759F35C26622900113757E00F8
:100FEC00C290C287C291D296D294D295C262227814
:100FFC008076070876070876010876040876FF08DD
:10100C0076FF08760B087602087601087601788C54
:10101C0076010876000876B40876FF0876FF087625
:10102C00FF0876030876FF0876010876FF08762518
:10103C000876D00876780876C80876040876FF0813
:10104C00760108760008767A087607087601087625
:10105C00010876000876FF227887E6FFC272BF038C
:0F106C0002D2727888C27DE630E102D27DC27E68
:10107B007889E630E102D27EC3EF94026008758E68
:10108B0001D273021096758E00C273227880E6141B
:10109B009000809378A4F67881E614900080937882
:1010AB00A5F67886E61490008D9378A6F6789FE6E1
:1010BB00F8700108C3E8941140027811E82828F56C
:1010CB006E256E256E28F56F256E2828F570789C99
:1010DB00E67538FF75390CB402067538A075390AF8
:1010EB00B4030675388275390578A3E61490009A17
:1010FB0093F569120FE622227896E6FA7897E6FBCB
:10110B007888E6B40305C3EB940EFB307F047A00BA
:10111B007BFFC3EB9AFCC3948250027C82757500F3
:10112B000575EC8575F0A4C3E5F0947D40F222D2F1
:10113B007F31031205697A007B007C1012055FE595
:10114B005F2AFA74003BFBDCF37C04C3EB13FBEA72
:10115B0013FADCF7FEC27F310322E5EF20E60375BD
:10116B0020000520903FFFE520146006901DFF1422
:10117B0060009304600375EF107597DE7597AD757E
:10118B0081C043FF8012055A75EF0075A900E5C7B2
:10119B00240420E70DF521E5B120E0068521C743A6
:1011AB00B101120FE67580FF75A48075F1C275D47D
:1011BB00BF75907475A57375F27B75D50475A60113
:1011CB0075E34075E201E4F8F6D8FD756B01120F7B
:1011DB00FB12166C78988676753001C2AF120573C8
:1011EB0012058312056912058A12056912059112FF
:1011FB00056912178F12057312057312056EC2AFB4
:10120B0078FA79FA308607D9FBD8F7021C001164FB
:10121B0011973102310378988676120FE675885054
:10122B0075891275C82475910475D84075A82275F7
:10123B00B80275E690759B80759D0075D1BC75BC29
:10124B005875BB0A75E88075B20112055AD2AF12F8
:10125B0008B353DACF207E0343DA20307E0343DA20
:10126B001043DA01C2D8C271120573D2617B037AC3
:10127B000CE55E70077A0CDB03021209120569207C
:10128B007003021209C270E55FC3940240E1E52FBF
:10129B00541F856160F561B560D5DAD5C26153DA4B
:1012AB00CF207E0343DA20307E0343DA10C2D8C24C
:1012BB007178A2E67008D274E52F54E0F52FC27551
:1012CB0075290012056E307409C3E529940A400292
:1012DB00D27512055F78023074027800C3E55F980F
:1012EB0040F0C2AF120583120583120583D2AF12F1
:1012FB000573754D0012055F788CE6C3940150039E
:10130B000213D6E530C3940150030213D620743573
:10131B00C3E55F94FF50030213D6C2AF120598D2F8
:10132B00AF12056EC3E55F940150EFC2AF12058398
:10133B00120564120583D2AF12056EC3E55F94FFED
:10134B0040E90218147F05D27F310312056EC2AF3C
:10135B00C27F3103AE5FC3E55F947FD2AF4076129D
:10136B00055AC2AF120598D2AFDFDC313AC3EE9407
:10137B00057897F61205731216AE1217977F0AD2DD
:10138B007F310312056EC2AFC27F3103AE5FC3E57F
:10139B005F947FD2AF50E612055AC2AF120583128B
:1013AB000564120583D2AFDFD6313AEE2405789669
:1013BB00F61205731216AE1217C612056E3103C361
:1013CB00E55F94FF50026118021814C3E55F954D59
:1013DB004003855F4D12056E78017988E7B40302EF
:1013EB007805C3E55F9840026100C2AF1205981201
:1013FB000598120598D2AF120573753000E4F531DC
:10140B00F5320531E531F470390532789AE6781901
:10141B00146012783214600D787D14600878FA1419
:10142B006003753200C3E53298401715327531B43D
:10143B0078998676C2AF120598D2AF7898867612D5
:10144B00056E120564E52A700530740241097801B6
:10145B002074027806C3E55F9840A712056EE52A53
:0F146B007003021209C2AF120FE6E4F522F52357
:10147A00F524F525F526F56AD2AF7885E6C333F566
:10148A0068E4F545F546F547F548F549F573F52C51
:10149A00F52DF53775730875BB1012055A120946F2
:1014AA00E5E820ECFBA8BDA9BEE97001F888741232
:1014BA00094A75730875BB107887E6FE76021164CF
:1014CA007887EEF6C2AF7564FF120A058522648535
:1014DA002265852266D2AF75220175240175250120
:1014EA0075260185636C756D017888E6B40307C2B9
:1014FA007D307602D27DD268D269753300120F4CE4
:10150A00120F71120A25120A2C120A25120A2C121B
:10151A000A2502152BC2AF1164D2AF75730075BBD1
:10152A000A120CB0120663120DCA120E14120A2CF9
:10153A00120C9F306D0312070320670312085630FE
:10154A00670312089D120DCA120E39120A2C120CC8
:10155A00B0306D0312073F120DCA120EB0120A2CD8
:10156A00120C9F306D0312079D120DCA120ED5126E
:10157A000A2C120CB0306D031207FA120DCA120FA0
:10158A004C120A2C120946120C9F120DCA120F7124
:10159A0012094A120A2C30692F206B2C8567648540
:1015AA00676585636C756D0179187A0CC3E53399A3
:1015BA004009C269D26A8A350215D2C3E55F94012D
:1015CA00400302152B02162C306A1B206B18E535D6
:1015DA00147004C26AA11FF535C3E55F9401400384
:1015EA0002152B02162C753600C3E56294014009D8
:1015FA0085676585636C756D01C3E56278FA9850F5
:10160A0021307404E52A601A78F0306B0585676426
:10161A007820C3E541985002A12B0536E55F6002A8
:10162A00C12F753600C2AF120FE67887E6FE760242
:10163A0011647887EEF6E4F522F523F524F525F50D
:10164A0026F568C268D2AF12055A120FE630740640
:10165A00E52A70024109788DE6C39401400241DD12
:10166A008108901A0D78201216F0E520B4A50CA373
:10167A001216F0E520B45A0302168E120FFB121648
:10168A00AE0216AD901A0378807B0A1216F0A308F0
:10169A00DBF9901A0F788C7B181216F0A308DBF985
:1016AA00901A2722C2AF12172F121709901A007424
:1016BA000E1216F5A374041216F5A374141216F575
:1016CA00901A0378807B0A1216F4A308DBF9901AA1
:1016DA000F788C7B181216F4A308DBF91217421242
:1016EA001720901A2722E493F622E6438F01538F9C
:1016FA00FD75EF0275B7A575B7F1F0538FFE22435A
:10170A008F02438F0175EF0275B7A575B7F1901A6D
:10171A000DF0538FFC22901A0D74A5D1F5901A0E74
:10172A00745AD1F5227A3079D07820901A40D1F0C3
:10173A00E520F709A3DAF7227A3079D0901A40E740
:10174A00D1F509A3DAF922AB77A878BB010279802F
:10175A00BB02027981BB03027982BB04027994BB82
:10176A0005027983BB06027986BB07027992BB0818
:10177A00027987BB0902799CBB0A027988BB0B02F2
:10178A007989E8F7227C05120573DCFB22C2AF12C5
:10179A00058312058A12059112059812056412052D
:1017AA008312058A1205911205981205641205839F
:1017BA0012058A120591120598D2AF22C2AF1205FC
:1017CA009812059112058A1205831205641205986A
:1017DA0012059112058A12058312056412059812E0
:1017EA00059112058A120583D2AF22AE77AF78C26D
:1017FA00AF120583120583120583120564DEF21205
:10180A000598120564DFF8D2AF2212179712178FC4
:10181A0012178F7577017578017579001217F57CA3
:10182A0005AD5F120573C3ED955F70F5C3E55F946F
:10183A0001400AC3E55F94FF403702185812175156
:10184A001216AE121797C2AF75EF1012178FDCD1AE
:10185A000579C3E5799403500280C112178F057880
:0F186A00E5771490009F93F808C3E57898500233
:1018790080A812178F12178F0577C3E577940C503C
:10188900028094120FFB1216AEC2AF75EF10121739
:011899008FBF
:0319FD000211656F
:101A00000E041407070104FFFF0B020101A55A0190
:101A100000B4FFFFFF03FF01FF25D078C804FF01DA
:081A200000FF07010100FFFFB8
:101A4000234638355F3341232020202020202020CA
:101A500023424C48454C492346383530232020202A
:101A60002020202020202020202020202020202076
:101C0000C2AFC2D37597DE7597AD7581C075A90057
:101C100043FF80752438752503B1C875EF0275E35D
:101C20004043F14053A4BF75D400D2867DFA7803B7
:101C300079E67C10752200752300901DD57B067512
:101C400024987525013086028145208608D8FBD965
:101C5000F9DCF781B7308608D8FBD9F9DCF781B712
:101C6000B188E493A3C39A6004DDC381B7DBDBB121
:101C70007A6002812E7B08E493FAA3B15BDBF87AE9
:101C800030B15B752200752300B17AEAFCEBFDC32D
:101C9000ED94FE400EB17A8A278B28ED30E0048A5D
:101CA000828B83B17A7AC270D8C3ED94FE601350F0
:101CB000CEBD0023EC60097520007521FF020000F5
:101CC0008100A827A9280809D804D90281D4B17EA7
:101CD000EAF281C80D81A3C3ED94035047EDA2E061
:101CE00092007AC5C3E5829400E583941C5092204B
:101CF0000010438F02438F0175B7A575B7F1F0301F
:101D0000001DA827A9280809438F01538FFDD80477
:101D1000D902A11FE275B7A575B7F1F0A3A10E53C3
:101D20008FFC817F7AC1BD030CE493A3FAB13FDC41
:101D3000F8B137817F8181AA22AB23B15BEBFAEA4C
:101D40006222752608C3E52313F523E52213F52245
:101D500050066323A0632201D526EAB1C8B1C87535
:101D6000260AEAF4200102D286300102C286B1C8F6
:101D7000C3134002C201D526EB22B17EEAFB2086C6
:101D800002A17E308602A183752608AE24AF25C34A
:101D9000EF13FFEE13FEB1CCB1C8C3EA13308602D5
:101DA0004480FA30E703632201C3E52313F523E5FA
:101DB0002213F52250066323A0632201D526D9E51C
:101DC0002265236523F52222AE24AF250E0FDEFE09
:101DD000DFFCD20122424C48656C6934373163F82C
:031DE000500601A9
:00000001FF
